S00600004844521B
S12301004FC6FFCE0032A700E701BD05E97E0777594F5552204E414D4500CE0108BD0486E3
S1230120BD0468CE01F0BD03ABCE01A2BD035B4FC6FFCE0032A700E701BD05E9D7319730BF
S1230140CE01F0BD04162022446F20796F752077616E7420746F206265207768697465206E
S12301606F7220626C61636B2000CE0148BD0486CE01A2BD0482BD0468CE01F0BD03AB4FA9
S12301805FD73197304F5FD73597344F5FD73797364F5FD73997384F5FD73B973A4F5FD77C
S12301A03D973C4F5FD73F973E4F5FD74197404F5FD7439742CE01F0BD04162020454E5497
S12301C045525041574E2020524F4F4B20204B4E49474854424953484F50515545454E206B
S12301E04B494E472020CE01F0BD03ABBD02F0D74597444FC6015849CB90890137364FC6A4
S12302000230EE003131A700E7014FC6025849CB90890137364FC60330EE003131A700E799
S1230220014FC6035849CB90890137364FC60430EE003131A700E7014FC6045849CB9089E8
S12302400137364FC60530EE003131A700E7014FC6055849CB90890137364FC60630EE00BD
S12302603131A700E7014FC6065849CB90890137364FC60430EE003131A700E7014FC60737
S12302805849CB90890137364FC60330EE003131A700E7014FC6085849CB90890137364FE1
S12302A0C60230EE003131A700E7014FC601D747974620215041574E524F4F4B20204B4EC7
S12302C049474854424953484F50515545454E204B494E4700CE02B4DF27CE01C2BD063B49
S12302E08602C671D72897273434BD0603CE01F04F36363636860536308D6F812027FA813A
S12303002D260E6C048D632436812027326D0027418030253D81092239A701A602E6035867
S123032049A702E703584958492527EB03A9022521EB018900251BA702E7036A0020C632A6
S12303408105270F3132336D04270440508200310C3931313131314F5F0D39C6208D0B2498
S123036006A700085A26F66F0039DF20DE22A6002709812C27048D020D3908DF22DE200C11
S1230380398620BDE1D139860DBDE1D1860ABDE1D13941100011434C4310000C434C491060
S12303A0000E434C52004A4F434C56863FBDE1D1BD0381DF22DF24C680BDE1AC810F260C01
S12303C09C24270C09A600BDE1D120ED811826178D07202A44454C2A0430EE003131BD0403
S12303E0428D0CDE2420CCA700810D26096F00860197267E03875D27C0085A20BC8620DF0A
S123040020DE22A7009626818022024C086F009726DF22DE2039DF24200486019726DE240B
S1230420DF22398DD896268407810126F6398DEEA600270B8D2F0820F78DC2D12622FA3932
S123044020BD8620BDE1D1862ABDE1D18644BDE1D18645BDE1D1864CBDE1D1862ABDE1D1B4
S1230460000F5345567EE1D18DC48DAE7E038736A60026046D0127068A308D836C016F0070
S12304803239C6202002C680A60027068DB2085A26F6394D2A0A36862D8DA53240508200F6
S12304A03434306F006F01C010822725046C0020F6CB1089278DB8C0E8820325046C0020EB
S12304C0F6CBE889038DA8C064820025046C0020F6CB648D9AC00A25046C0020F8CB0A8D2E
S12304E08EE7006C018D883131393736E601375FA6002A075C3040600082003637C610377D
S123050030A6042A094060058200A7046C014F5F660266032404EB05A904465666026603DA
S12305206A0026F04D26115D260EA602E6036601242540508200201F660124126303630228
S123054053436C0326086C022604CB018900972BD72CE603A6020D31313131313139373648
S1230560E601375FA6002A075C30406000820036373430E6034D26065D26030D204F6D04CF
S12305802A0A6004600524026A046C0186016D022B0B4C680369022B04811126F5A700A6E2
S12305A004E6056F046F05E003A2022407EB03A9020C20010D69056904640266036A0026A2
S12305C0E6A604E60566012404405082003131313131313937C60837305F58492404EB011C
S12305E089006A0026F4313139A60148AB00E60158495849EB01A900CB1989364456A70013
S1230600E70139DE27DF29309629A702962AA7033930EE02395F6D002704085C20F84F3919
S123062030EE028DF05D276609A600088120265E095A20F1C6808D056F0039C620DF29DE93
S123064027A60008DF27DE29A7002704085A26ED3930EE02DF27378DBC1733273110232E8B
S12306604CDE27200330EE02DF274D27216D00272E4A27030820F65D27258D2A20142095AA
S123068030EE025D2708A6002704085A20F5DF276F0030EE00313131316E00C68020073000
S12306A0EE0220EAC620A6008D084D2712085A26F517DF29DE27A700270108DF27DE2939D7
S12306C08DEF4F20EDDE276F0020EFC601D72FDF278DAB5D272AD72CDE208DA2D72BD62CCE
S12306E0D12B23035F4F39DE27DF29DE20DF2DDE29A60008DF29DE2DA1002608085A26EDCA
S1230700D62F4F39DE2008DF207C002FD62B5A20CBDF27DE20A600270F08DF20DE27E60080
S12307202704081127EB0C39DE276D0026F80D39368D24DE27DF22328D2CDE22DF276F00F7
S1230740200ADF298D11DE29DF228D1736962B9726DE2DDF2232399626972B7F0026DE22CB
S1230760DF2D397E02F07E0493F70111B70110FE0110A600E60139CE01F0BD0416201257E6
S123078048415420495320594F5552204E414D4500CE077FBD0486BD0468CE01F0BD03AB1E
S12307A0CE01A2BD035BCE01F0BD04162022444F20594F552057414E5420544F204245203D
S12307C05748495445204F5220424C41434B2000CE07AEBD0486CE01A2BD0482BD0468CEC1
S12307E001F0BD03ABCE01F0BD035B4F5FD7319730CE00348C01002705A7000820F6C601FB
S1230800D747B601F08142270686FF97469747CE01F0BD04162020454E54455220313D4CB1
S12308204F4E472047414D452C20303D53484F52542047414D4500CE0817BD0486BD0468B6
S1230840CE01F0BD03ABBD02F0D7459744CE0192C6024FA700E7015CA702E7035CA704E7E0
S1230860055CA706E7075CA708E709C604A70AE70B5AA70CE70D5AA70EE70FC601D749C65D
S123088008D74BC601D74DC608D74FD649964DBD09914FA700A701D649C00827037E08C0FD
S12308A0D64DBD099FE60137D649964DBD09913396478101270750A700E70120034F20F70D
S12308C0D649C00727037E08D8D649964DBD0991D6479646A700E701D649C00227037E0834
S12308E0F4D649964DBD0991D647964640508200A700E701D649C00127037E091FD64DBD7D
S1230900099FE60137D649964DBD099133964781FF270986FF50A700E70120034F20F7D631
S12309204DCB01D74DD04F2E037E088BD649CB01D749D04B2E037E0883C601BD099F4FC674
S123094064A700E70108088601C6F4A700E70108088601C62CA700E70108088601C645A75F
S123096000E70108088603C684A700E70108088607C6D0A700E701D647C00126037E098643
S1230980BD09CFBD09C6BD09CFBD09CC7E098009825858581B4897FFC601D7FEDEFE39586F
S12309A0CB908601D7FF97FEDEFE397E09DB7E09EA7E0A467E0BB87E0F527E10E07E1136DD
S12309C07E11A37E11F57E12477E15B97E16807E1A5F7E1BE37E1D327E1E45D649964DBD46
S12309E00991E6012A01507E09F0D653965520EF5817581B16CBBC8601D7FF97FEDEFE4FC1
S1230A00B701EAB701EBB701ECA600B701E6A601B701E7A602B701E8A603B701E9A60481A2
S1230A2020270CB701EAA60581202703B701EB86CE91FF2707A600B701ED2005864EB70196
S1230A40ED4FB701EE39D635DB5927037E0BB34F975B975ABD09D2D65B965ACBAF8900D014
S1230A605F925E2C037E0BB3D637C00126037E0B0DD6618608BD0991E601C1FE27037E0BB6
S1230A800DD6FFC004D7FFDEFEE6012604E60327037E0B0DC601D749C608D74BC601D74D7E
S1230AA0C608D74FD649964DBD0991E6012E037E0AD2D661D753C606D755BD09B4D6512653
S1230AC0037E0B0DC607D755BD09B4D65126037E0B0DD64DCB01D74DD04F2E037E0AA4D6BB
S1230AE049CB01D749D04B2E037E0A9CD6618605BD09914FA700A701A706A70786FFC6FEF2
S1230B00A702E703C6FAA704E7057E0BA9D63127037E0BB3D6618601BD0991E601C0FE2767
S1230B20037E0BB3E6032608E6052604E60727037E0BB3C601D749C608D74BC601D74DC66B
S1230B4008D74FD649964DBD0991E6012E037E0B71D661D753C603D755BD09B4D6512603D8
S1230B607E0BB3C604D755BD09B4D65126037E0BB3D64DCB01D74DD04F2E037E0B43D649EB
S1230B80CB01D749D04B2E037E0B3BD6618601BD09914FA700A701A708A70986FFC6FAA757
S1230BA004E705C6FEA706E707C601D7355FD751D75039C601D751399649905327172A01D5
S1230BC040D64DD055270E2A01501127081B80032F037E0F4AD649585858DB4D588601D7ED
S1230BE0FF97FEDEFEE6012A0150C10126037E0C40C10226037E0D54C10326037E0D33C133
S1230C000426037E0E28C10526037E0F11C10626037E0F28CE01F0BD041620182A2A2A2A47
S1230C202A2A426F617264204572726F722A2A2A2A2A2A00CE0C1CBD0486BD04687EE0E3A7
S1230C40D64DD0552A0150D767C0012F037E0F4AD653585858DB55588601D7FF97FEDEFE3E
S1230C60E601D765D649585858DB4D588601D7FF97FEDEFEE601D04727037E0CD8D649D05F
S1230C8053C10126037E0C92C10226037E0CAF7E0F4AD667C00126037E0CA5D66527037EC1
S1230CA00F4A7E0F44D66526037E0F4A7E0F44D66727037E0F4AD649C00727037E0F4AD6FF
S1230CC0FFC010D7FFDEFEE60127037E0F4AD66527037E0F4A7E0F44D653D049C10126036D
S1230CE07E0CEDC10226037E0D0A7E0F4AD667C00126037E0D00D66527037E0F4A7E0F4462
S1230D00D66526037E0F4A7E0F44D66727037E0F4AD649C00227037E0F4AD6FFCB10D7FF1D
S1230D20DEFEE60127037E0F4AD66527037E0F4A7E0F44D649D0532A0150964D90552A012E
S1230D4040C0022F037E0F4A80022EF91B81FF26F47E0F44D649D05326037E0DC7D64DD0A5
S1230D605527037E0F4AD649D0532A0150C00126037E0F44D649D0532F037E0D8CD653C02D
S1230D8001D765D649CB01D7697E0D98D649C001D765D653CB01D769D669D751D665D76B8F
S1230DA0D651585858DB4D588601D7FF97FEDEFEE60127037E0F4AD651CB01D751D06B2E46
S1230DC0037E0DA07E0F44D64DD0552A0150C00126037E0F44D64DD0552F037E0DEDD65575
S1230DE0C001D767D64DCB01D76D7E0DF9D64DC001D767D655CB01D76DD66DD751D667D75D
S1230E006BD649585858DB51588601D7FF97FEDEFEE60127037E0F4AD651CB01D751D06BAC
S1230E202E037E0E017E0F44D649D0532A0150964D90552B01401B27037E0F4AD649D053D0
S1230E402A0150C00126037E0F44D649D0532F037E0E7AD649CB01D765D653C001D769D6B7
S1230E604DD0552F037E0E71D64DCB01D7677E0E9ED64DC001D7677E0ED7D653CB01D765C0
S1230E80D649C001D769D64DD0552F037E0E98D655C001D7677E0ED7D655CB01D767C60107
S1230EA0D751D669D065CB01D76BD665585858DB67588601D7FF97FEDEFEE60127037E0F3B
S1230EC04A7C00657C0067D651CB01D751D06B2E037E0EAA7E0F444FC601D751D669D065C0
S1230EE0CB01D76BD665585858DB67588601D7FF97FEDEFEE60127037E0F4A7C00657A00F2
S1230F0067D651CB01D751D06B2E037E0EE47E0F44D649D0532A0150964D90552B01401B92
S1230F2026037E0E3C7E0D54D649D0532A0150C0012F037E0F4AD64DD0552A0150C0012FA3
S1230F40037E0F4A5FD751D750394FC601D751975039C601D751D63B27037E1042CE01F0B5
S1230F60BD041620204B494E47532053494445204F5220515545454E532053494445202856
S1230F804B2F512900CE0F65BD0486BD0468CE01F0BD03ABCE01E6BD035BCE01E68602C6AA
S1230FA071D7289727BD06A4BD06C5DE27DF2020024B00CE0FB1BD069BCE0271BD07112479
S1230FC0037E0FFDD63927037E1076D66F8601BD0991E6032608E6052604E60727037E104F
S1230FE0AA4FA700A701A708A709C606E705A704C602E707A706C601D73B7E102FD63D27B0
S1231000037E1076D66F8605BD0991E6032604E60527037E10AA4FA700A701A706A707C67F
S123102002E703A702C606E705A704C601D73BD63F963ECB018900D73F973E4F5FD7519745
S12310405039CE01F0BD04162022594F55204841564520414C5245414459204D4F5645442D
S123106020594F5552204B494E472000CE104ABD0486BD046839CE01F0BD04162022594F43
S123108055204841564520414C5245414459204D4F56454420594F555220524F4F4B20000C
S12310A0CE107EBD0486BD046839CE01F0BD04162024544845524520415245204F43435593
S12310C0504945442053515541524553204245545745454E2000CE10B2BD0486BD04683923
S12310E0CE0110DFFEC601D765C608D771C601D767C608D773DEFE0808DFFEA601810627DC
S1231100037E110CD665D76FD667D77581FA27037E111BD665D761D667D777D667CB01D7F6
S123112067D0732E037E10F5D665CB01D765D0712E037E10ED39D649964DBD0991A600E6FF
S123114001DFF4D7799778D6539655BD0991A600E601DFF6D77B977AD653D77DD655D77F2A
S1231160D649D781D64DD783DEF4A600E601DEF6A700E701DEF44FA700A701BD09C3D67D69
S1231180D753D67FD755D681D749D683D74DDEF4D6799678A700E701DEF6D67B967AE701D1
S12311A0A70039BD09BAD661D753D677D755CE0110DFECC601D749C608D74BC601D74DC6BF
S12311C008D74FDEEC0808DFECE6012E037E11DABD09B4D65126037E11F4D64DCB01D74D57
S12311E0D04F2E037E11C3D649CB01D749D04B2E037E11BB39BD09BAD66FD753D675D75509
S1231200CE0110DFECC601D749C608D74BC601D74DC608D74FDEEC0808DFECE6012D037E30
S1231220122CBD09B4D65126037E1246D64DCB01D74DD04F2E037E1215D649CB01D749D0E9
S12312404B2E037E120D39CE0110DFF0C601D7494FC608D74BC601D74DC608D74FDEF008AF
S123126008DFF0E6012E037E12C5CE0110DFF2C601D753C608D785C601D755C608D787DE5E
S1231280F20808DFF2E6012F037E12ABBD09B4D6519650C001820026065D26037E12ABBDAF
S12312A009BDD651C00126037E12EBD655CB01D755D0872E037E127FD653CB01D753D085AA
S12312C02E037E1277D64DCB01D74DD04F2E037E125DD649CB01D749D04B2E037E1255D670
S12312E041C00126037E16A57E19C8CE01F0BD0416202557484552452049532054484520F4
S1231300504945434520594F552057414E5420544F204D4F56452000CE12F3BD0486CE01C9
S1231320A2BD0482BD0468CE01F0BD03ABBD02F0D74D974CBD02F0D7499748C00A27037E9B
S12313401358D641C00126037E1587BD09B7D651C00126037E12EB39D649964DBD0991DF89
S1231360F0E6012F037E139ACE01F0BD041620185448455245204953204E4F205355434823
S12313802050494543452000CE1370BD0486CE01A2BD0482BD04687E12EBD6492FF9C008A4
S12313A02F037E12EBD64D2FEEC0082F0220E8BD09ABCE01F0BD0416200B4D4F5645205959
S12313C04F55522000CE13BABD0486CE01E6BD0482200A20544F20574845524500CE13D3DD
S12313E0BD0486BD0468CE01F0BD03ABBD02F0D7559754BD02F0D7539752D6532F04C008A3
S12314002F037E12EBD6552F04C0082F037E12EBD6539655BD0991DFF2E6012F037E142A37
S1231420BD09B4D65126037E145DCE01F0BD04162019544841542049534E27542041204C9D
S12314404547414C204D4F56452000CE1432BD0486CE01A2BD0482BD04687E12EBBD09BDC2
S1231460D651C00126037E149ECE01F0BD0416201B594F552043414E2754204D4F56452075
S1231480494E544F20434845434B2000CE1471BD0486CE01A2BD0482BD04687E12EBCE01AF
S12314A0F0BD04162009414343455054454400CE14A6BD0486BD0468DEF2E60126037E1495
S12314C0EBBD09AECE01F0BD04162010594F552043415054555245204D592000CE14CCBD61
S12314E00486CE01E6BD0482BD0468DEF0A600E601DEF2A700E7014FDEF0A700A701D63F02
S1231500CB01D73FDEF2E601C00627037E1513C601D73BE601C00227037E1536D64DC00838
S123152027037E1529C601D73DD64DC00127037E1536C601D739D653C00126037E1547C08B
S12315400726037E154739DEF2E601C00127037E1546DEF24FC605A700E701CE01F0BD04D0
S1231560162018414E442050524F4D4F54455320544F204120515545454E00CE1563BD04E4
S123158086BD04687E1546CE01F0BD0416201E594F552043414E275420434153544C452085
S12315A04F5554204F4620434845434B00CE158FBD0486BD04687E12EBD635C00126037E2C
S12315C01610D649D06127037E1610D649D05326037E1610D64DD0772E037E15F2D64DC0B1
S12315E00826037E15F2D6899688CB788900D7899788D64DD0772D037E1610D64DC0012621
S1231600037E1610D6899688CB648900D7899788D653D06F2A0150965590752A01401B977B
S123162079CE0032BD05E916019679544426FCDB899988D7899788D653585858DB5558865F
S123164001D7FF97FEDEFEE601C0FF27037E166FD653C00126037E1660C00727037E166F70
S1231660CE019AA600E601DB899988D7899788390000000000000000000000000000000033
S1231680BD09C04F9741974097599758D651C00126037E1699C601D759BD09BDD651C00143
S12316A026037E16C2CE01F0BD0416200F49204841564520574F4E20494E2000CE16AD7E5B
S12316C01A0686D8C6F0D75F975E4F975D975C978B978ACE0110DFFAC601D78DC608D78F17
S12316E0C601D791C608D793DEFA0808DFFAE6012D037E181FCE0110DFFCC601D795C60837
S1231700D797C601D799C608D79BDEFC0808DFFCE6012C037E1805D68DD749D691D74DD686
S123172095D753D699D755BD09B4D651C00126037E1805DEFCA600E601D79D979CDEFAA699
S123174000E601D79F979E4F975D975CD69D26037E1768D69D58CB90860197FED7FFDEFE30
S1231760A600E601D75D975CDEFC969ED69FA700E701DEFA4FA700A70197899788BD09BA6A
S1231780BD1F07D65D965CDB899988D75D975CBD09C0D651C00126037E17B2DEFCD69D96D0
S12317A09CA700E701DEFAD69F969EA700E7017E18054FC601D78B978A975B975ABD09D23B
S12317C0D65D965CDB5B995AD75D975CDEFCD69D969CA700E701DEFAD69F969EA700E70172
S12317E0D65F965ED05D925C2D037E1805D65D965CD75F975ED68DD7A1D691D7A3D695D788
S1231800A5D699D7A7D699CB01D799D09B2E037E170AD695CB01D795D0972E037E1702D6A4
S123182091CB01D791D0932E037E16E8D68DCB01D78DD08F2E037E16E0D68B26037E19B85F
S1231840BD09B1D651C00126037E1869CE01F0BD041620094920434153544C4500CE1854DF
S1231860BD0486BD04687E1A5ED6A1D749D6A3D74DD6A5D753D6A7D755BD09ABCE01F0BD8F
S12318800416200B49204D4F5645204D592000CE1884BD0486CE01E6BD0482200520544FE8
S12318A02000CE189DBD0486D6559654BD04932004202C2000CE18B1BD0486D6539652BD95
S12318C00493BD0468D653585858DB5558D7FDDEFCE60126037E1901BD09AECE01F0BD0441
S12318E016200F414E442054414B4520594F55522000CE18E3BD0486CE01E6BD0482BD042F
S123190068D649585858DB4D58D7FBDEFAA600E601DEFCA700E701DEFA4FA700A701D65375
S1231920C00126037E192EC00727037E196BDEFCE601C1FF27037E196B86FFC6FBA700E780
S123194001CE01F0BD04162019414E4420492050524F4D4F544520544F20412051554545BD
S12319604E00CE1949BD0486BD0468D6A1D06127037E19B8D635C00126037E198CDEFCE67C
S123198001C0FA27037E198CC601D735D631C00126037E19A2D6A3C00127037E19A2C601DA
S12319A0D731D637C00126037E19B8D6A3C00827037E19B8C601D737D68B27037E1A25D628
S12319C059C00126037E19EACE01F0BD04162015495427532041205354414C454D4154453C
S12319E020494E2000CE19D0201CCE01F0BD04162011594F55204841564520574F4E204994
S1231A004E2000CE19F2BD0486D63F963EBD04932007204D4F56455300CE1A12BD0486BD28
S1231A2004687EE0E3BD09C3D651C00126037E1A5ECE01F0BD04162015414E4420594F55AA
S1231A402041524520494E20434845434B00CE1A39BD0486BD04684FC601D741974039CEB8
S1231A6001F0BD0416BD046ACE01F0BD041620252020202D2D2D2D2D2D2D2D2D2D2D2D2DEB
S1231A802D2D2D2D2D2D2D2D2D2D2D2D2D2D2D2D2D2D2D2D00CE1A70BD0486BD0468C60828
S1231AA0D749C601D74BD6499648BD0493CE1B46BD0486CE1B46BD0486BD042EC601D74D02
S1231AC0C608D74FD649964DBD0991DFF0E60127037E1AEACE01F0BD0416200549202020EF
S1231AE000CE1ADCBD0486BD042EDEF0E60196472A01505D2D037E1B20BD09ABCE01F0BDA8
S1231B0004162003492000CE1B04BD0486CE01EDBD048220022A00CE1B15BD0486BD042E68
S1231B20DEF0E60196472A01505D2E037E1B51BD09ABCE01F0BD0416CE1B04BD0486CE0112
S1231B40EDBD048220022000CE1B46BD0486BD042ED64DCB01D74DD04F2E037E1AC4CE011C
S1231B60F0BD0416200449202000CE1B66BD0486BD0468CE01F0BD0416CE1A70BD0486BD3C
S1231B800468D649C001D749D04B2D037E1AA6CE01F0BD0416202320202020203120202042
S1231BA03220202033202020342020203520202036202020372020203800CE1B97BD0486A7
S1231BC0BD0468FE01F0BD0416BD046A39203800CE1BB0BD0486BD0468FE01F0BD0416BDCA
S1231BE0046A39CE0110DFF0C601D7A9C608D7ABC601D7ADC608D7AFDEF00808DFF0E601C2
S1231C002E037E1D17CE0110DFF2C601D7B1C608D7B3C601D7B5C608D7B7DEF20808DFF226
S1231C20E6012F037E1CFDD63FC0042C037E1C39D645C00126037E1C42DEF2E60126037ED6
S1231C401CFDD6A9D749D6ADD74DD6B1D753D6B5D755BD09B4D651C00126037E1CFDDEF2C7
S1231C60E601A600D7B997B8DEF0E601A600D7BB97BAD6BB96BADEF2A700E7014FDEF0A7B2
S1231C8000A701BD09C3D651C00026037E1CE986D8C6F0D7BD97BCBD09D5D6BD96BCC0F051
S1231CA082D82D0826035D27037E1CB14F97BD97BCD6B926037E1CD45058CB908601D7FF1A
S1231CC097FEDEFEA600E60140508200DBBD99BCD7BD97BCD6BD96BCD05B925A2D037E1C56
S1231CE0E9D6BD96BCD75B975AD6B996B8DEF2A700E701D6BB96BADEF0A700E701D6B5CB1F
S1231D0001D7B5D0B72E037E1C1AD6B1CB01D7B1D0B32E037E1C12D6ADCB01D7ADD0AF2E0B
S1231D20037E1BF8D6A9CB01D7A9D0AB2E037E1BF039CE0110DFF4C601D7BFC608D7C1C697
S1231D4001D7C3C608D7C5DEF40808DFF4E6012D037E1E2ACE0110DFF6C601D7C7C608D72A
S1231D60C9C601D7CBC608D7CDDEF60808DFF6E6012E037E1E10D6BFD749D6C3D74DD6C72F
S1231D80D753D6CBD755BD09B4D651C00126037E1E10DEF6A600E601D7CF97CEDEF4A6002D
S1231DA0E601D7D197D0D6D196D0DEF6A700E7014FDEF4A700A70197899788BD09BABD09C4
S1231DC0C94F97D397D2BD09D8D6CF58CB90860197FED7FFDEFEA600E601DBD399D2DB8946
S1231DE09988D7D397D2D0BD92BC2D0526065D26037E1DFCD6D396D2D7BD97BCD6CF96CE54
S1231E00DEF6A700E701D6D196D0DEF4A700E701D6CBCB01D7CBD0CD2E037E1D69D6C7CBA4
S1231E2001D7C7D0C92E037E1D61D6C3CB01D7C3D0C52E037E1D47D6BFCB01D7BFD0C12EDC
S1231E40037E1D3F39CE0110DFEEC601D7D5C608D7D7C601D7D9C608D7DBDEEE0808DFEE2D
S1231E60E6012E037E1EECCE0110DFF8C601D7DDC608D7DFC601D7E1C608D7E3DEF808081C
S1231E80DFF8E6012D037E1ED2D6D5D749D6D9D74DD6DDD753D6E1D755BD09B4D651C00122
S1231EA026037E1ED2DEF8E60150860158CB9097FED7FFDEFEA600E60140508200D7E59707
S1231EC0E4D0D392D22D037E1ED2D6E596E4D7D397D2D6E1CB01D7E1D0E32E037E1E7CD620
S1231EE0DDCB01D7DDD0DF2E037E1E74D6D9CB01D7D9D0DB2E037E1E5AD6D5CB01D7D5D0A1
S1231F00D72E037E1E5239BD09C9CE0110DFE6C601D749C608D74BC601D74DC608D74FDEC7
S1231F20E60808DFE6E6012E037E1F7DCE0110DFE8C601D753C608D785C601D755C608D757
S1231F4087DEE80808DFE8E6012F037E1F63BD09B4D651C001270CBD09BDD651C001260317
S1231F607E1FB5D655CB01D755D0872E037E1F41D653CB01D753D0852E037E1F39D64DCB19
S1231F8001D74DD04F2E037E1F1FD649CB01D749D04B2E037E1F17D641C001260CD6899602
S11B1FA088CBD08907D7899788D6899688CBF48901D7899788392C0346
S50300F606
S9030100FB
